:100074009307000063880700372500001305455DDA
:100084006F20C05A67800000974100009381415F50
:100094001385C18017660000130686E13306A64067
:1000A40093050000EF20C0321725000013054558C2
:1000B40063080500172500001305C551EF200057FC
:1000C400EF2040270325010093054100130600009B
:1000D400EF0050716F20C022130101FF232481001F
:1000E40083C741812326110063920702930700000E
:1000F400638A0700374500001305859A97000000BE
:10010400E700000093071000238AF1808320C100D8
:10011400032481001301010167800000930700009C
:10012400638E0700B745000037450000938585E9D5
:100134001305859A1703000067000000678000001C
:10014400130101FF2326810013040101B7470000B6
:1001540083A747E89387870003A7070023A6E180C6
:1001640083A7C18093F7170093B7170093F7F70F8E
:10017400138507000324C1001301010167800000F7
:10018400130101FF2326810013040101B747000076
:1001940083A747E89387870003A7070023A6E18086
:1001A40003A7C180B7070100B377F70093B717001F
:1001B40093F7F70F138507000324C100130101010E
:1001C40067800000130101FE232E81001304010245
:1001D4002326A4FEB747000083A747E89387870038
:1001E40003A7070023A6E18083A7C18093F7170024
:1001F40063900702B747000083A747E89387470047
:100204000327C4FE23A0E700930700006F008000CB
:100214009307F0FF138507000324C10113010102B2
:1002240067800000130101FF2326810013040101EC
:10023400B747000083A747E89387870003A7070011
:1002440023A6E18003A7C180B7070100B377F700B5
:10025400639A0700B747000083A747E883A707000E
:100264006F0080009307F0FF138507000324C1008B
:100274001301010167800000130101FE232E110008
:10028400232C8100130401022326A4FE6F00000323
:10029400130000008327C4FE83C7070013850700EB
:1002A400EFF05FF2130705009307F0FFE304F7FE96
:1002B4008327C4FE938717002326F4FE8327C4FEF6
:1002C40083C70700E39607FC930700001385070024
:1002D4008320C1010324810113010102678000000E
:1002E400130101FD232611022324810213040103B7
:1002F400232EA4FC232CB4FC232604FE032784FD14
:100304009307100063C6E700930700006F0080099D
:10031400EFF05FF12324A4FE032784FE9307F0FF8C
:10032400E308F7FE8327C4FE138717002326E4FEA1
:10033400138707008327C4FDB387E700032784FEE0
:100344001377F70F2380E70013000000032584FED2
:10035400EFF05FE7130705009307F0FFE308F7FEEC
:10036400832784FD9387F7FF0327C4FE6350F702B6
:10037400032784FE9307A000630CF700032784FE81
:100384009307D0006306F7006FF09FF81300000096
:100394008327C4FE0327C4FDB307F70023800700A7
:1003A4008327C4FE138507008320C102032481022E
:1003B4001301010367800000130101FC232E1102C5
:1003C400232C8102130401042326A4FC2320B4FC5F
:1003D4002322C4FC232404FE232204FE832744FC9A
:1003E40063DC07021306000093060000032504FCE7
:1003F400832544FC3307A64013080700333806015D
:10040400B387B640B3860741938706002320E4FCF4
:100414002322F4FC232204FE832704FC032744FC48
:10042400B3E7E7006390070A832784FE1387170066
:100434002324E4FE138707008327C4FCB387E70063
:10044400130700032380E7006F00C00B032704FC9D
:10045400832744FC1306A00093060000130507003D
:1004640093850700EF10C06113070500938705000B
:100474001377F70F832784FE938617002324D4FE73
:10048400938607008327C4FCB387D70013070703A9
:100494001377F70F2380E700032704FC832744FC2A
:1004A4001306A000930600001305070093850700B8
:1004B400EF10801513070500938705002320E4FC43
:1004C4002322F4FC832744FCE342F0F8832744FC12
:1004D40063960700832704FCE39A07F6832744FE08
:1004E40063820702832784FE138717002324E4FE14
:1004F400138707008327C4FCB387E7001307D002E0
:100504002380E700232604FE6F00C006832784FEB1
:100514001387F7FF8327C4FEB307F7402320F4FEB5
:100524008327C4FE0327C4FCB307F70083C707006F
:10053400A30FF4FC832704FE0327C4FC3307F7004E
:100544008327C4FE8326C4FCB387F6000347070051
:100554002380E700832704FE0327C4FCB307F700C6
:100564000347F4FD2380E7008327C4FE9387170025
:100574002326F4FE832784FE13D7F701B307F7007D
:1005840093D71740138707008327C4FEE3C0E7F817
:10059400832784FE0327C4FCB307F70023800700E6
:1005A400832784FE138507008320C103032481036A
:1005B4001301010467800000130101FB2326810459
:1005C400130401052326A4FC2320B4FC2322C4FC29
:1005D4002324D4FC93070700A30FF4FA232404FE76
:1005E4006F000009832704FC93F7F700232EF4FC23
:1005F4000327C4FD9307900063C4E7028327C4FD67
:1006040013F7F70F832784FE8326C4FCB387F60011
:10061400130707031377F70F2380E7006F004002E7
:100624008327C4FD13F7F70F832784FE8326C4FCB6
:10063400B387F600130777051377F70F2380E700D6
:10064400832744FC9397C701032704FC13584700EE
:1006540033E80701832744FC93D84700232004FD93
:10066400232214FD832784FE938717002324F4FE9A
:10067400832704FC032744FCB3E7E700E39407F66D
:100684006F004002832784FE138717002324E4FEAF
:10069400138707008327C4FCB387E7000347F4FBF1
:1006A4002380E700032784FE832784FCE34CF7FCC4
:1006B400232604FE6F00C006832784FE1387F7FFFA
:1006C4008327C4FEB307F7402322F4FE8327C4FE26
:1006D4000327C4FCB307F70083C70700A301F4FE94
:1006E400832744FE0327C4FC3307F7008327C4FE93
:1006F4008326C4FCB387F600034707002380E70082
:10070400832744FE0327C4FCB307F700034734FEE2
:100714002380E7008327C4FE938717002326F4FE73
:10072400832784FE13D7F701B307F70093D7174045
:10073400138707008327C4FEE3C0E7F8832784FEFA
:100744000327C4FCB307F70023800700832784FE34
:10075400138507000324C104130101056780000009
:10076400130101FD2326810213040103232EA4FC9B
:10077400232CB4FC232604FE232404FE9307100038
:100784002322F4FE6F00C0088327C4FD83C707003B
:100794002320F4FE032704FE9307F00263D2E70448
:1007A400032704FE9307900363CCE702032784FE28
:1007B4009307070093972700B387E70093971700E1
:1007C40013870700832704FEB307F700938707FD09
:1007D4002324F4FE930710002326F4FE6F00800206
:1007E4008327C4FE639E0702032704FE9307D002F7
:1007F400631AF7009307F0FF2322F4FE9307100017
:100804002326F4FE8327C4FD93871700232EF4FCCC
:100814008327C4FD83C70700E39807F66F008000B1
:1008240013000000032784FE832744FEB307F70266
:100834002324F4FE832784FD63880700832784FD33
:100844000327C4FD23A0E700832784FE1385070044
:100854000324C1021301010367800000130101FD99
:100864002326810213040103232EA4FC232CB4FCAD
:10087400232604FE232404FE6F00000E8327C4FDF8
:1008840083C707002322F4FE032744FE9307F002E4
:1008940063DAE702032744FE9307900363C4E70285
:1008A400930710002326F4FE832784FE1397470042
:1008B400832744FEB307F700938707FD2324F4FE40
:1008C4006F00C008032744FE9307000663DAE702BB
:1008D400032744FE9307600663C4E70293071000EE
:1008E4002326F4FE832784FE13974700832744FEC0
:1008F400B307F700938797FA2324F4FE6F000005EB
:10090400032744FE9307000463DAE702032744FE47
:100914009307600463C4E702930710002326F4FEE0
:10092400832784FE13974700832744FEB307F70009
:10093400938797FC2324F4FE6F0040018327C4FEB1
:1009440063940702930710002326F4FE8327C4FD53
:1009540093871700232EF4FC8327C4FD83C7070065
:10096400E39E07F06F00800013000000832784FDDE
:1009740063880700832784FD0327C4FD23A0E700C1
:10098400832784FE138507000324C1021301010396
:1009940067800000130101FD232681021304010373
:1009A400232EA4FC232CB4FC8327C4FD2326F4FEAD
:1009B4006F0000018327C4FD93871700232EF4FCE6
:1009C4008327C4FD83C70700E39607FE6F00400238
:1009D400032784FD93071700232CF4FC8327C4FD0D
:1009E40093861700232ED4FC034707002380E700D7
:1009F400832784FD83C70700E39C07FC8327C4FD8A
:100A0400238007000327C4FD8327C4FEB307F740F0
:100A1400138507000324C10213010103678000004A
:100A2400130101FD2326810213040103232EA4FCD8
:100A3400232CB4FC232AC4FC232604FE6F000005E7
:100A44008327C4FD13871700232EE4FC03C7070084
:100A5400832784FD93861700232CD4FC83C70700C7
:100A64006306F700930710006F0000048327C4FE99
:100A7400938717002326F4FE0327C4FE832744FD2F
:100A84006346F700930700006F0000028327C4FD4C
:100A940083C7070063880700832784FD83C7070093
:100AA400E39007FA93070000138507000324C102AB
:100AB4001301010367800000130101FE232E81004E
:100AC400130401022326A4FEB7E7F50513870710D4
:100AD4008327C4FE3347F702B747000083A747E8DC
:100AE4009387070123A0E7009307000013850700FD
:100AF4000324C1011301010267800000130101EC0A
:100B0400232E1112232C8112232A2113232831137B
:100B140023264113232451131304011483A70181B1
:100B240093F707FF232AF4FC232C04FC6F00801F97
:100B3400832744FD13890700930900009307C4EC3D
:100B44001307000393068000930509001386090028
:100B540013850700EFF05FA61307C4ECB727000066
:100B64009385C77113050700EFF0DFE2232E04FC21
:100B74006F00000C832744FD2326F4FC0327C4FDE7
:100B8400832744FD3307F70083A70181637EF700C1
:100B94001307C4ECB72700009385077213050700F9
:100BA400EFF05FDF6F0000068327C4FD0327C4FC5A
:100BB400B307F70083C70700138A0700930A0000EE
:100BC400930744EC130700039306200093050A00DF
:100BD40013860A0013850700EFF01F9E130744ECE9
:100BE400B72700009385477213050700EFF09FDADB
:100BF400130744EC9307C4EC93050700138507001F
:100C0400EFF05FD90327C4FD93077000631CF7005E
:100C14001307C4ECB72700009385877213050700F8
:100C2400EFF05FD78327C4FD93871700232EF4FCCE
:100C34000327C4FD9307F000E3DEE7F21307C4ECD7
:100C4400B72700009385C77213050700EFF09FD400
:100C5400232E04FC6F000008832744FD2328F4FCA2
:100C64008327C4FD032704FDB307F70003C7070068
:100C74009307F00163FAE7028327C4FD032704FD09
:100C8400B307F70003C707009307E00763EEE70025
:100C94008327C4FD032704FDB307F70083C70700B8
:100CA4002300F4EC6F00C0009307E0022300F4EC8F
:100CB400A30004EC130704EC9307C4EC93050700AA
:100CC40013850700EFF01FCD8327C4FD938717001A
:100CD400232EF4FC0327C4FD9307F000E3DEE7F6BC
:100CE4001307C4ECB72700009385077313050700A7
:100CF400EFF05FCA9307C4EC13850700EFF0CFD77A
:100D0400832744FD93870701232AF4FC832744FDAA
:100D140093F7F70F63800702832784FD93871700F7
:100D2400232CF4FC032784FD9307F000E3D2E7E0CF
:100D34006F00800013000000B7270000138547737D
:100D4400EFF08FD3032744FD23A8E18013000000B4
:100D54008320C1130324811303294113832901131D
:100D6400032AC112832A811213010114678000002F
:100D7400130101FB232611042324810423222105CA
:100D84002320310513040105EF0080772320A4FEFE
:100D94002322B4FE232604FE6F008011B72700002F
:100DA4001385077BEFF04FCDB7470000138707A3E8
:100DB4008327C4FE93972700B307F70083A7070090
:100DC40013850700EFF04FCBB7470000138787A0C8
:100DD4008327C4FE93972700B307F70083A7070070
:100DE400E7800700232CA4FC232EB4FC032784FDF6
:100DF4008327C4FD930604FB9305070013860700AD
:100E040013850600EFF04FDB930704FB13850700FF
:100E1400EFF08FC6B72700001385477BEFF0CFC5EF
:100E24000327C4FD930740063307F702832784FD95
:100E340093060000B387D702B306F700032784FDA7
:100E4400930740063306F702B339F7021309060085
:100E5400B387360193890700032604FE832644FEE4
:100E64001305090093850900EF1080061307050098
:100E740093870500232CE4FC232EF4FC032784FD34
:100E84008327C4FD930604FB93050700138607001C
:100E940013850600EFF04FD2930704FB1385070078
:100EA400EFF08FBD8327C4FE938717002326F4FE3B
:100EB4000327C4FE93079000E3D2E7EEB7270000B0
:100EC40013854773EFF04FBB130000008320C10468
:100ED4000324810403294104832901041301010526
:100EE40067800000130101FE232E1100232C8100D2
:100EF40013040102B7470000938707EB2322F4FE93
:100F0400B7570000938707EB2320F4FE232404FE45
:100F1400EF00006E232604FE6F000004832744FEC6
:100F2400138747002322E4FE03A70700832704FE58
:100F3400938647002320D4FE83A707003307F702D4
:100F4400832784FEB307F7002324F4FE8327C4FE1B
:100F5400938717002326F4FE0327C4FE9307F03F6C
:100F6400E3DEE7FAEF008069EFF09FE0EF0040680E
:100F7400130000008320C101032481011301010235
:100F840067800000130101FF232611002324810040
:100F940013040101B72700001385877BEFF0CFAD61
:100FA400B72700001385877DEFF00FADB72700004A
:100FB4001385C77FEFF04FACB73700001385478226
:100FC400EFF08FABB737000013858785EFF0CFAA1A
:100FD400130000008320C1000324810013010101D8
:100FE40067800000130101E72326111823248118C8
:100FF4002322211923203119232E4117232C511781
:10100400232A611723287117232681172324911774
:101014002322A1172320B11713040119232EA4E6B8
:10102400232CB4E6B70700F02324F4FCB70700F040
:10103400938707012322F4FCB7C701001385072017
:10104400EFF09FA7232004FC232E04FAEF00C049ED
:101054001309050093890500EF00804A1307050072
:101064009387050013064006930600001305070046
:1010740093850700EF00D0651307050093870500EB
:1010840013060700938607001305090093850900DA
:10109400EF0010641307050093870500232CE4FA7E
:1010A400EFF00F8A930705006388070AEF00C04337
:1010B400930704E8130700039306800013860500D2
:1010C4009305050013850700EFF00FCF930704E89D
:1010D40013850700EFF04F9AB73700001385078791
:1010E400EFF08F99EF00C041930704E81307000362
:1010F40093068000138605009305050013850700F9
:10110400EFF08FCB930704E813850700EFF0CF9639
:10111400B737000013850787EFF00F96832784FB0A
:10112400138A070093D7F741938A0700930704E8CB
:1011340093050A0013860A0013850700EFF0CFA772
:10114400930704E813850700EFF00F93B737000007
:1011540013854787EFF04F92EFF08F8293070500D6
:10116400E38C07FE930704E89305F00F138507004B
:10117400EFF00F9713000000B7370000138587873F
:10118400EFF08F8F930704E813850700EFF0CF8EFD
:10119400B727000013854773EFF00F8E130704E899
:1011A40013064000B73700009385C787130507006F
:1011B400EFF01F879307050063960700EFF09FDCAD
:1011C4006F004031034704E89307C0066316F70035
:1011D400EFF01FBA6F000030034704E8930740079D
:1011E4006316F700EFF01FD06F00C02E034704E82A
:1011F40093072006631CF702930704E893872700EC
:101204009305000013850700EFF08FD5232EA4F873
:101214008327C4F96358F0000325C4F9EFF0DF898C
:101224006F00402BEFF01FD66F00C02A034704E87D
:1012340093074006631AF702930704E8938727008D
:101244009305000013850700EFF04FE12320A4FA73
:10125400832704FA6356F000032704FA23A8E180E5
:10126400EFF0DF896F000027034704E89307700756
:10127400631CF70A930704E893872700130744F8CD
:101284009305070013850700EFF04FDD2326A4FA2A
:10129400832744F8130744F89305070013850700D0
:1012A400EFF0CFDB2324A4FA832744F8130744F890
:1012B4009305070013850700EFF04FDA2322A4FA01
:1012C400032744FA93071000631CF7008327C4FA2A
:1012D400032784FA1377F70F2380E7006F00801F3A
:1012E400032744FA93072000631EF7008327C4FAF8
:1012F400032784FA13170701135707412390E700C4
:101304006F00401D032744FA93074000631AF70057
:101314008327C4FA032784FA23A0E7006F00801B05
:10132400EFF05FC66F00001B034704E89307200734
:101334006312F71A232604FC930704E89387270013
:10134400130704F89305070013850700EFF00FD186
:10135400232AA4FA832704F8130704F89305070043
:1013640013850700EFF08FCF2328A4FA032704FB8B
:10137400930710006310F702832744FB83C7070019
:101384002326F4FCB737000013854788EFE0DFEE2F
:101394006F008005032704FB930720006310F70206
:1013A400832744FB839707002326F4FCB737000008
:1013B4001385C788EFE05FEC6F000003032704FB8D
:1013C400930740006310F702832744FB83A70700B9
:1013D4002326F4FCB737000013854789EFE0DFE9E3
:1013E4006F008000EFF01FBA032704FB930710007F
:1013F400630EF700032704FB930720006308F7003C
:10140400032704FB930740006316F70C832744FB70
:10141400138B070093D7F741938B0700930704E8D6
:10142400130700039306800093050B0013860B003B
:1014340013850700EFF04F98930704E8138507001E
:10144400EFE09FE3B73700001385C789EFE0DFE2E1
:101454008327C4FC138C070093D7F741938C0700B0
:10146400930704E893050C0013860C00138507000A
:10147400EFE09FF4930704E813850700EFE0DFDF54
:10148400B73700001385078AEFE01FDF8327C4FC0A
:10149400138D070093D7F741938D0700832704FB2F
:1014A40093961700930704E81307000393050D00B0
:1014B40013860D0013850700EFF00F90930704E8DF
:1014C40013850700EFE05FDBB73700001385478A19
:1014D400EFE09FDA13000000EFE09FC693070500DA
:1014E400E38C07FE6FF09FB6F32500C8732500C098
:1014F40067800000F31500C8731500C06780000002
:10150400F32520C8732520C067800000F31520C888
:10151400731520C067800000F32500CA732500C23C
:1015240067800000F31500CA731500C267800000CD
:10153400F32510CA732510C267800000F31510CA82
:10154400731510C267800000F32520CA732520C2DA
:1015540067800000F31520CA731520C2678000005D
:10156400F32530CA732530C267800000F31530CAF2
:10157400731530C267800000F32540CA732540C24A
:1015840067800000F31540CA731540C267800000ED
:10159400F32550CA732550C267800000F31550CA62
:1015A400731550C267800000F32560CA732560C2BA
:1015B40067800000F31560CA731560C2678000007D
:1015C400F32570CA732570C267800000F31570CAD2
:1015D400731570C267800000F32580CA732580C22A
:1015E40067800000F31580CA731580C2678000000D
:1015F400F31500CC731500C467800000F31510CCFC
:10160400731510C46780000013030500138E0500D2
:101614009308000063DC0500B337A000330EB0402C
:10162400330EFE403303A0409308F0FF63DC060052
:10163400B337C000B306D04093C8F8FFB386F64072
:101644003306C040130706001308030093070E0077
:10165400639C0628B73500009385858A6376CE0E91
:10166400B70601006378D60C9336061093C61600AD
:10167400939636003355D600B385A50083C505007F
:1016840013050002B386D500B305D540630CD5001D
:10169400B317BE00B356D3003317B600B3E7F60052
:1016A4003318B3009355070133DEB702131607014D
:1016B40013560601B3F7B70213050E003303C6032E
:1016C4009396070193570801B3E7D70063FE6700B9
:1016D400B387E7001305FEFF63E8E70063F66700DE
:1016E4001305EEFFB387E700B387674033D3B70230
:1016F4001318080113580801B3F7B702B3066602BA
:10170400939707013368F80093070300637CD800BC
:10171400330807019307F3FF6366E8006374D80096
:101724009307E3FF131505013365F50093050000E6
:101734006F00000E3705000193060001E36CA6F26A
:10174400930680016FF01FF363140600730010000A
:10175400B7070100637AF60C9336061093C6160099
:1017640093963600B357D600B385F50083C70500BA
:10177400B387D70093060002B385F6406390F60C56
:10178400B307CE409305100013530701B3DE67027D
:10179400131607011356060193560801B3F767029F
:1017A40013850E00330ED60393970701B3E7F600B3
:1017B40063FEC701B387E7001385FEFF63E8E70014
:1017C40063F6C7011385EEFFB387E700B387C7410C
:1017D40033DE67021318080113580801B3F76702D0
:1017E400B306C603939707013368F80093070E0006
:1017F400637CD800330807019307FEFF6366E800A3
:101804006374D8009307EEFF131505013365F500E3
:10181400638A0800B337A000B305B040B385F54030
:101824003305A04067800000B7070001930600015C
:10183400E36AF6F2930680016FF0DFF23317B60025
:10184400B356FE0013550701331EBE00B357F30011
:10185400B3E7C70133DEA6021316070113560601C8
:101864003318B300B3F6A6023303C60393950601F7
:1018740093D60701B3E6B60093050E0063FE660037
:10188400B386E6009305FEFF63E8E60063F66600B0
:101894009305EEFFB386E600B386664033D3A60213
:1018A4009397070193D70701B3F6A602330666029E
:1018B40093960601B3E7D7009306030063FEC700BF
:1018C400B387E7009306F3FF63E8E70063F6C70016
:1018D4009306E3FFB387E70093950501B387C740F9
:1018E400B3E5D5006FF05FEA6366DE18B707010061
:1018F40063F4F60413B706101347170013173700E1
:10190400B7370000B3D5E6009387878AB387B7005B
:1019140083C70700B387E70013070002B305F74046
:101924006316F70213051000E3E4C6EF3335C30072
:10193400134515006FF0DFEDB70700011307000131
:10194400E3E0F6FC130780016FF09FFB3357F600CA
:10195400B396B600B366D7003357FE00331EBE00FD
:10196400B357F300B3E7C70113DE0601335FC703C0
:1019740013980601135808013316B6003377C703CA
:10198400B30EE8031315070113D707013367A70044
:1019940013050F00637ED7013307D7001305FFFF3C
:1019A4006368D7006376D7011305EFFF3307D700C9
:1019B4003307D741B35EC7039397070193D7070152
:1019C4003377C7033308D80313170701B3E7E700D6
:1019D40013870E0063FE0701B387D7001387FEFF4A
:1019E40063E8D70063F607011387EEFFB387D700D8
:1019F40013150501B70E01003365E5009386FEFF5C
:101A04003377D500B3870741B376D6001358050161
:101A140013560601330ED702B306D8023307C702A2
:101A24003308C8023306D70013570E013307C70023
:101A34006374D7003308D80193560701B3860601AF
:101A440063E6D702E394D7CEB70701009387F7FF85
:101A54003377F70013170701337EFE003313B30007
:101A64003307C70193050000E374E3DA1305F5FFB8
:101A74006FF0DFCB93050000130500006FF05FD912
:101A8400138E05001308000063DC0500B337A000C3
:101A9400B305B040338EF5403305A0401308F0FF82
:101AA40063DA0600B337C000B306D040B386F6400D
:101AB4003306C040930806009307050093050E0003
:101AC40063940624373700001307878A6376CE0EA3
:101AD400B70601006378D60C9336061093C6160039
:101AE400939636003353D600330767000347070045
:101AF4003307D700930600023383E640638CE60085
:101B0400B3156E003357E500B3186600B365B7002C
:101B1400B317650093D6080133D7D502139508018E
:101B240013550501B3F5D5023307A7021396050132
:101B340093D50701B3E5C50063FAE500B385150144
:101B440063E6150163F4E500B3851501B385E5404B
:101B540033D7D5029397070193D70701B3F5D5027D
:101B64003307A70293950501B3E7B70063FAE700CB
:101B7400B387170163E6170163F4E700B38717011E
:101B8400B387E74033D5670093050000630A080074
:101B9400B337A000B305B040B385F5403305A0408A
:101BA400678000003703000193060001E36C66F2CE
:101BB400930680016FF01FF3631406007300100096
:101BC400B70601006372D60A9336061093C6160050
:101BD40093963600B355D6003307B7000347070082
:101BE4003307D700930600023383E6406398E60880
:101BF4003307CE4093D508013356B7021395080135
:101C04001355050193D607013377B7023306A602AD
:101C14001317070133E7E600637AC7003307170198
:101C2400636617016374C700330717013307C7409E
:101C3400B356B7029397070193D707013377B702D7
:101C4400B386A60213170701B3E7E70063FAD700C8
:101C5400B387170163E6170163F4D700B38717014D
:101C6400B387D7406FF01FF2B70500019306000158
:101C7400E362B6F6930680016FF0DFF5B3186600F1
:101C8400B356EE00B3156E003357E500B317650085
:101C940013D508013367B700B3D5A602139E080114
:101CA400135E0E01B3F6A602B385C50313960601AF
:101CB40093560701B3E6C60063FAB600B38616016D
:101CC40063E6160163F4B600B3861601B386B64024
:101CD40033D6A6021317070113570701B3F6A6025A
:101CE4003306C603939606013367D700637AC700A9
:101CF40033071701636617016374C70033071701BD
:101D04003307C7406FF01FEFE362DEE837070100D7
:101D140063FCE60413B706101347170013173700C4
:101D2400B738000033D3E6009388888AB388680004
:101D340003C308003303E30013070002B30867403A
:101D4400631E670263E4C601636CC5003306C540C5
:101D5400B306DE40B335C500B385B640930706002D
:101D6400138507006FF09FE2B70800011307000115
:101D7400E3E816FB130780016FF09FFAB357660080
:101D8400B3961601B3E6D70033576E0093DE06010F
:101D9400B35FD703B3151E01139E0601135E0E0134
:101DA400B3576500B3E5B70093D7050133161601A1
:101DB400331515013377D703330FFE0313170701C8
:101DC400B3E7E70013870F0063FEE701B387D7008B
:101DD4001387FFFF63E8D70063F6E7011387EFFF7C
:101DE400B387D700B387E74133DFD7039395050162
:101DF40093D50501B3F7D703330EEE039397070189
:101E0400B3E5F50093070F0063FEC501B385D50064
:101E14009307FFFF63E8D50063F6C5019307EFFF5F
:101E2400B385D50013170701B70F01003367F70017
:101E3400B385C541138EFFFFB377C701935E0601D7
:101E440013570701337EC601338FC703330EC7030D
:101E5400B387D7033307D703B38EC70193570F0153
:101E6400B387D70163F4C7013307F70113DE070112
:101E74003307EE00370E0100130EFEFFB3F7C70160
:101E840093970701337FCF01B387E70163E6E5004A
:101E9400639EE500637CF5003386C740B3B7C70093
:101EA400B387D7003307F74093070600B307F5401D
:101EB4003335F500B385E540B385A540339365001C
:101EC400B3D717013365F300B3D515016FF01FCCF9
:101ED4001303050093880500130706001308050083
:101EE4009387050063920628B73500009385858A99
:101EF40063F6C80EB70601006378D60C9336061055
:101F040093C61600939636003355D600B385A500C4
:101F140083C5050013050002B386D500B305D5407B
:101F2400630CD500B397B800B356D3003317B6008B
:101F3400B3E7F6003318B3009355070133D3B70260
:101F44001316070113560601B3F7B702130503006E
:101F5400B30866029396070193570801B3E7D700C5
:101F640063FE1701B387E7001305F3FF63E8E70097
:101F740063F617011305E3FFB387E700B38717413F
:101F8400B3D8B7021318080113580801B3F7B702FE
:101F9400B3061603939707013368F8009387080084
:101FA400637CD800330807019387F8FF6366E80071
:101FB4006374D8009387E8FF131505013365F500B2
:101FC40093050000678000003705000193060001B7
:101FD400E36CA6F2930680016FF01FF3631406000E
:101FE40073001000B70701006370F60C93360610F7
:101FF40093C6160093963600B357D600B385F50002
:1020040083C70500B387D70093060002B385F64063
:102014006396F60AB387C8409305100093580701E6
:1020240033DE1703131607011356060193560801EE
:10203400B3F7170313050E003303C6039397070181
:10204400B3E7F60063FE6700B387E7001305FEFFFE
:1020540063E8E70063F667001305EEFFB387E70064
:10206400B387674033D317031318080113580801C3
:10207400B3F71703B3066602939707013368F800B2
:1020840093070300637CD800330807019307F3FF29
:102094006366E8006374D8009307E3FF1315050132
:1020A4003365F50067800000B7070001930600015F
:1020B400E364F6F4930680016FF01FF43317B6005F
:1020C400B3D6F80013550701B357F3003318B30020
:1020D40033D3A60213160701B398B80013560601AA
:1020E400B3E71701B3F6A602B30866029395060197
:1020F40093D60701B3E6B6009305030063FE160109
:10210400B386E6009305F3FF63E8E60063F6160181
:102114009305E3FFB386E600B3861641B3D8A6025F
:102124009397070193D70701B3F6A6023306160364
:1021340093960601B3E7D7009386080063FEC700B1
:10214400B387E7009386F8FF63E8E70063F6C70008
:102154009386E8FFB387E70093950501B387C740EB
:10216400B3E5D5006FF09FEB63E6D518B707010020
:1021740063F4F60413B70610134717001317370058
:10218400B7370000B3D5E6009387878AB387B700D3
:1021940083C70700B387E70013070002B305F740BE
:1021A4006316F70213051000E3EE16E13335C3009E
:1021B4001345150067800000B707000113070001ED
:1021C400E3E0F6FC130780016FF09FFB3357F60042
:1021D400B396B600B366D70033D7F800B398B80007
:1021E400B357F300B3E7170193D80601B35E17039F
:1021F40013980601135808013316B60033771703F2
:10220400330ED8031315070113D707013367A7004B
:1022140013850E00637EC7013307D7001385FEFFC5
:102224006368D7006376C7011385EEFF3307D700D1
:102234003307C741335E17039397070193D7070109
:10224400337717033308C80313170701B3E7E7000D
:1022540013070E0063FE0701B387D7001307FEFFC1
:1022640063E8D70063F607011307EEFFB387D700CF
:1022740013150501370E01003365E5009306FEFFD3
:102284003377D500B3870741B376D60013580501D9
:1022940013560601B308D702B306D8023307C702A0
:1022A4003308C8023306D70013D708013307C70021
:1022B4006374D7003308C80193560701B386060137
:1022C40063E6D702E39ED7CEB70701009387F7FFF3
:1022D4003377F70013170701B3F8F8003313B3008B
:1022E4003307170193050000E37EE3CC1305F5FFE4
:1022F4006FF01FCD930500001305000067800000F8
:10230400130101FF930500002324810023261100FB
:1023140013040500EF008019B747000003A507E880
:102324008327C50363840700E780070013050400BF
:10233400EF00C03A130101FF23248100232021016F
:1023440037440000374900009307C49F1309C99F0D
:102354003309F940232611002322910013592940FF
:10236400630009021304C49F93040000832704003C
:102374009384140013044400E7800700E31899FED3
:1023840037440000374900009307C49F130949A04C
:102394003309F94013592940630009021304C49F07
:1023A400930400008327040093841400130444005E
:1023B400E7800700E31899FE8320C100032481000D
:1023C40083244100032901001301010167800000F7
:1023D4001303F00013070500637EC3029377F7002D
:1023E4006390070A63920508937606FF1376F60056
:1023F400B386E6002320B7002322B7002324B700C6
:102404002326B70013070701E366D7FE631406000B
:1024140067800000B306C34093962600970200002D
:10242400B38656006780C6002307B700A306B7002B
:102434002306B700A305B7002305B700A304B7001C
:102444002304B700A303B7002303B700A302B70014
:102454002302B700A301B7002301B700A300B7000C
:102464002300B7006780000093F5F50F939685006D
:10247400B3E5D50093960501B3E5D5006FF0DFF61B
:102484009396270097020000B386560093820000BB
:10249400E78006FA93800200938707FF3307F7402B
:1024A4003306F600E378C3F66FF0DFF3130101FDA2
:1024B400B7470000232C410103AA07E82320210386
:1024C4002326110203298A14232481022322910240
:1024D400232E3101232A510123286101232671016E
:1024E4002324810163000904130B0500938B050069
:1024F400930A10009309F0FF832449001384F4FF26
:102504006342040293942400B304990063840B048B
:1025140083A74410638077051304F4FF9384C4FFF6
:10252400E31634FF8320C102032481028324410281
:10253400032901028329C101032A8101832A41015C
:10254400032B0101832BC100032C81001301010320
:10255400678000008327490083A644009387F7FF20
:10256400638E870423A20400E38806FA832789186C
:1025740033978A00032C4900B377F700639207026C
:10258400E78006000327490083278A146314870120
:10259400E38427F9E38807F8138907006FF0DFF570
:1025A4008327C91883A544083377F700631C070001
:1025B40013050B00E78006006FF0DFFC232289007F
:1025C4006FF09FFA13850500E78006006FF09FFB0C
:1025D400130101FF23248100B747000037440000A2
:1025E400938747A0130484A03304F440232291006A
:1025F4002326110093542440638004021304C4FF6F
:102604003304F400832704009384F4FF1304C4FF09
:10261400E7800700E39804FE8320C10003248100BF
:102624008324410013010101678000009305050024
:102634009306000013060000130500006F0040001D
:10264400B747000003A707E883278714638C0704B0
:1026540003A747001308F001634EE8061318270088
:1026640063060502338307012324C30883A887185C
:10267400130610003316E600B3E8C80023A41719A4
:102684002324D310930620006304D50213071700F4
:1026940023A2E700B387070123A4B70013050000B2
:1026A400678000009307C7142324F7146FF05FFAC0
:1026B40083A6C7181307170023A2E700B3E6C600D2
:1026C40023A6D718B387070123A4B7001305000076
:1026D400678000001305F0FF678000009308D005B1
:1026E40073000000634405006F000000130101FF44
:1026F40023248100130405002326110033048040A1
:10270400EF00C000232085006F000000B7470000E1
:0827140003A587E867800000BF
:10271C002020000020202000200000002D200000A0
:10272C0020207C007C0A00000A0D0000746F74618C
:10273C006C2020203A2000006164642F73756220A5
:10274C003A2000006D756C20202020203A200000DB
:10275C0064697620202020203A2000006C64202020
:10276C00202020203A2000007374202020202020DC
:10277C003A2000006A6D7020202020203A200000B2
:10278C006A202020202020203A200000616C7569EE
:10279C00202020203A200000616C75202020202071
:1027AC003A2000000A0000002C20000020206420A9
:1027BC003C616464723E202D2D20646973706C61E1
:1027CC0079206D656D6F7279200A000020206220DF
:1027DC003C62617564726174653E202D2D207365B9
:1027EC0074206261756472617465200A00000000D7
:1027FC00202072203C616464723E203C77696474D2
:10280C00683E202D2D2072656164206D656D6F72A0
:10281C007920776F72640A00202077203C61646411
:10282C00723E203C76616C75653E203C7769647421
:10283C00683E202D2D207772697465206D656D6F53
:10284C00727920776F72640A00000000202020202B
:10285C0077696474683D312C2032206F7220340A01
:10286C00000000003A0000003E3E00000A0D3A0055
:10287C0068656C7020000000636861722040000085
:10288C0073686F7274204000696E74204000000001
:10289C00203D200028000000290A0D000001020242
:1028AC0003030303040404040404040405050505DC
:1028BC0005050505050505050505050506060606B8
:1028CC00060606060606060606060606060606069C
:1028DC000606060606060606060606060707070788
:1028EC00070707070707070707070707070707076C
:1028FC00070707070707070707070707070707075C
:10290C00070707070707070707070707070707074B
:10291C000707070707070707070707070808080837
:10292C00080808080808080808080808080808081B
:10293C00080808080808080808080808080808080B
:10294C0008080808080808080808080808080808FB
:10295C0008080808080808080808080808080808EB
:10296C0008080808080808080808080808080808DB
:10297C0008080808080808080808080808080808CB
:10298C0008080808080808080808080808080808BB
:0C299C00080808080808080808080808CF
:1039A8001000000000000000037A5200017C0101B1
:1039B8001B0D0200100000001800000048DCFFFF8B
:1039C8007804000000000000100000002C00000037
:1039D800ACE0FFFF500400000000000010000000F1
:1039E80040000000E8E4FFFF300400000000000091
:0439F80000000000CB
:0839FC0074000000200100002E
:043A0400DC000000E2
:103A0800041500001C150000341500004C150000BA
:103A1800641500007C15000094150000AC1500002A
:103A2800C4150000DC1500003827000044270000FA
:103A3800502700005C27000068270000742700005A
:103A4800802700008C27000098270000A42700008A
:103A580000000000443D0000AC3D0000143E0000A2
:103A6800000000000000000000000000000000004E
:103A7800000000000000000000000000000000003E
:103A8800000000000000000000000000000000002E
:103A9800000000000000000000000000000000001E
:103AA800000000000000000000000000000000000E
:103AB80000000000000000000000000000000000FE
:103AC80000000000000000000000000000000000EE
:103AD80000000000000000000000000000000000DE
:103AE80000000000000000000000000000000000CE
:103AF80000000000000000000100000000000000BD
:103B08000E33CDAB34126DE6ECDE05000B00000081
:103B1800000000000000000000000000000000009D
:103B2800000000000000000000000000000000008D
:103B3800000000000000000000000000000000007D
:103B4800000000000000000000000000000000006D
:0C3E8000583A0000000100F0583A000021
:040000030000008C6D
:00000001FF
